:020000040000FA
:020000000728CF
:04000A00003400348A
:02000E000730B9
:100010009F008316D73081008B0180308600FF302F
:10002000850083128601142805181428851A2728AC
:10003000051A362852203530860052203930860085
:1000400052203A30860052207630860014288518D7
:100050003828452035308600452039308600452037
:100060003A308600452076308600142885182928E5
:1000700045207630860045203A30860045203930CC
:1000800086004520353086001428193005197D304A
:1000900085190A30A1008930A000A00B4D28A10BC2
:1000A0004B280800FA30A1008930A000A00B562888
:0E00B000A10B54281430A200A20B5C280800FB
:02400E00413F30
:00000001FF
